:100000000C944B050C94B6050C9457080C94B6054B
:100010000C94B6050C94B6050C94B6050C94B60574
:100020000C94B6050C94B6050C94CF150C94B6053B
:100030000C9482230C94B6050C94B6050C94B6056A
:100040000C94B6050C94B6050C94B6050C94B60544
:100050000C94B6050C94D7230C94B6050C94B605F5
:100060000C94B6050C94B6050C94B6050C94B60524
:100070000C94B6050C94B6050C94B6050C94B60514
:100080000C94B6050C94B6050C94B6050C94B60504
:100090000C94B6050C94B605D609D809E409E40910
:1000A000E409E409E409E409DA09DC09DE09E40900
:1000B000E409D809E609E409E409A009D609E40934
:1000C000E409DC09E409E409E409E409E409E409D0
:1000D000DE09D609C209E409C609E409E409E4090C
:1000E000A209DA09E409E409D009E409E409E40908
:1000F000A409E209E409C409E409D809E409E40906
:10010000D409C809E409CA09DC09E409E409E409D5
:10011000D209CC09E409E409E409E409E409E409A1
:10012000E409CE09E409A609E409E409DA09E409C5
:10013000E409E209E409E409E409E409E409E40959
:10014000E409E409E409A809E409E409E409D00997
:10015000E409E409E409E409E409E409E409E40937
:10016000E409E409AA09E409AC09AE09E409E409CF
:10017000E409B009B209B409E409B609B809E40907
:10018000E409E409E009BA09E409BE09BC09C009A7
:10019000E409E409E409E409E2090A0A180A240A5C
:1001A000240AFC09240A240A240A240A240A240A08
:1001B000240A240A240A240A240A240A240AFE09F6
:1001C000240A000A240A240A240A240A1C0A240AEB
:1001D000330A1A0A240A240A240A240A240A240AAA
:1001E000240A240A240A240A240A240A240AF409D0
:1001F000100A020A140A240A040A240A080A240A11
:10020000120A060A160A0C0A0E0A240A240A240AEA
:10021000240A240A240A240AF609F809FA091E0AFB
:10022000200A240A240A240A220AB10AC70AD50A83
:10023000E30A030B1A0B3D0B5A0BE20B0F0CA60C37
:10024000430D290D8D0DA20DAD0DB30DB80DBD0DD6
:10025000C20DE30D1A1441143915411439158D14CA
:10026000B01439150715161599199919C319C31919
:100270001E1A491C491C491C521A491C3D1B3D1B96
:10028000031C491C181C361C807B46010203763A6D
:10029000687F6577482B353B6978796439141E3C53
:1002A0006A7A1D16041A1F3D6B061B070821203EA3
:1002B0006C2C19091715223F6D11050B0A1C2340E0
:1002C0006E7E100D182425416F360E0C1227264223
:1002D0007037380F33132D43717534322F2E44721B
:1002E0007C7D28303174457351504A524D492A540F
:1002F00066594F5C5F4C4B4E62635A5D5E6029539A
:1003000067585B56576147554842403E3C3A3B452B
:100310006843413F3D2B357E697A790078141E7C15
:100320006A7B1D16041A1F7F6B061B070821204DD0
:100330006C2C19091715224A6D11050B0A1C234C48
:100340006E49100D182425516F360E0C1227264FBA
:100350007037380F33132D52717534502F2E4E7263
:10036000397D283065314B735464586776012A779C
:100370003259745C5F66024662635A5D5E6029535F
:1003800044575B565561470380291E1F20212223B5
:10039000242526272D2E2A2B141A0815171C180C75
:1003A00012132F302878041607090A0B0D0E0F338D
:1003B000343579311D1B06190511103637387D5536
:1003C0007A2C393A3B3C3D3E3F4041424353475FE4
:1003D0006061565C5D5E57595A5B626346483244C1
:1003E00045677B7F650301025250514F68696A6B14
:1003F0006C6D6E6F7071725800494C754A4D734B3D
:100400004E767C777E7466547225303258200062B6
:1004100025303458200077253032582000214353AE
:10042000335F4630210A00214353335F46305F4536
:100430005252210A00214353335F46305F4F5652D8
:10044000210A00214353335F5245414459210A0098
:10045000214353335F455252210A00214353335FF6
:100460004F5652210A00214353325F45305F4630D8
:10047000210A00214353325F4630210A00214353B1
:10048000325F4530210A00214353325F494E4954BF
:10049000210A00214353325F455252210A00214371
:1004A00053325F4F5652210A00214353315F45308A
:1004B0005F25303258210A00214353315F455252A3
:1004C000210A00214353315F494E56210A004C2531
:1004D000752000532575200049443A2530345828AA
:1004E0002564290A004D6F7573653A206E6F74207C
:1004F000737570706F727465640A000A4552523ADF
:10050000253032580A0052257520005725752000E5
:10051000572575200057257520005825752000495E
:1005200025752000696E69740A000A4552523A2501
:100530003032580A000A4B6579626F617264207329
:10054000746172742E0A000A55534220636F6E66FE
:100550006967757265642E0A000A0A544D4B3A6445
:10056000613163613361622F4C5546410A0A0034A0
:1005700003490042004D0020005000430020006B62
:10058000006500790062006F006100720064002065
:100590000063006F006E00760065007200740065F5
:1005A00000720000000E0374002E006D002E006B20
:1005B000002E000000040309040902740004010075
:1005C000A03209040000010301010009211101000A
:1005D000012240000705810308000A090401000107
:1005E00003000000092111010001223600070582E5
:1005F0000308000A09040200020300000009211197
:1006000001000122220007058303200001070503E2
:100610000320000109040300010300000009211167
:100620000100012239000705840320000112011096
:100630000100000008EDFEEE1B01000102000105B3
:10064000010906A101050719E029E7150025019513
:1006500008750181020508190129059505750191A3
:10066000029501750391010507190029F715002569
:100670000195F875018102C00631FF0974A10109D5
:1006800075150026FF009520750881020976150072
:1006900026FF00952075089102C005010980A1017F
:1006A00085021601002637001A81002AB70075104E
:1006B00095018100C0050C0901A101850316010007
:1006C000269C021A01002A9C02751095018100C027
:1006D00005010906A101050719E029E71500250113
:1006E00095087501810295017508810105081901B8
:1006F000290595057501910295017503910105077D
:10070000190029FF150026FF00950675088100C015
:10071000636F6E73756D65723A20253034580A0028
:1007200073797374656D3A20253034580A000A00D5
:100730002530325820006B6579626F6172643A200F
:10074000004C45443A20253032580A0025303258B2
:100750003A202530386225730A00722F6320303129
:100760003233343536370A0064656C5F6B65795F08
:100770006269743A2063616E27742064656C3A2064
:10078000253032580A006164645F6B65795F626985
:10079000743A2063616E2774206164643A202530C6
:1007A00032580A003F00433E20004C25640A000AEC
:1007B000092D20436F6E736F6C65202D0A455343DE
:1007C0002F713A09717569740A000A092D204D616B
:1007D000676963202D0A643A0964656275670A785F
:1007E0003A096465627567206D61747269780A6B95
:1007F0003A096465627567206B6579626F6172643E
:100800000A6D3A096465627567206D6F7573650AD4
:10081000763A0976657273696F6E0A733A09737472
:10082000617475730A633A09636F6E736F6C652048
:100830006D6F64650A302D343A096C6179657230E8
:100840002D34284631302D4634290A506175733ACB
:1008500009626F6F746C6F616465720A6E3A094E5B
:100860004B524F0A003F004E4B524F3A206F666684
:100870000A004E4B524F3A206F6E0A0074696D6544
:10088000725F72656164333228293A202530346CF6
:10089000580A006B6579626F6172645F6E6B726F8C
:1008A0003A2025580A006B6579626F6172645F694E
:1008B000646C653A2025580A006B6579626F617235
:1008C000645F70726F746F636F6C3A2025580A0012
:1008D000686F73745F6B6579626F6172645F6C657A
:1008E000647328293A2025580A000A092D205374D8
:1008F00061747573202D0A004743433A20352E3426
:100900002E30204156522D4C4942433A20322E304F
:100910002E30204156525F415243483A2061767250
:1009200035310A004F5054494F4E533A204C5546EA
:10093000412045585452414B455920434F4E534F47
:100940004C4520434F4D4D414E44204E4B524F207D
:100950004B45594D41505F53454354494F4E2042FA
:100960004F4F544C4F414445525F53495A450A003A
:100970004255494C443A20646131636133616220DD
:100980002832333A33343A353220417072203236CD
:100990002032303230290A005649443A2030784615
:1009A00045454428742E6D2E6B2E29205049443A1B
:1009B000203078316265652849424D205043206BD4
:1009C0006579626F61726420636F6E7665727465BB
:1009D0007229205645523A203078303030310A00A2
:1009E000444553433A20636F6E76657274204942E2
:1009F0004D205043206B6579626F61726420746F83
:100A0000205553420A000A092D2056657273696FFA
:100A10006E202D0A000A6D6F7573653A206F666649
:100A20000A000A6D6F7573653A206F6E0A000A6BD3
:100A30006579626F6172643A206F66660A000A6BBC
:100A40006579626F6172643A206F6E0A000A6D61A7
:100A5000747269783A206F66660A000A6D61747272
:100A600069783A206F6E0A000A64656275673A20F9
:100A70006F6E0A000A64656275673A206F66660ADF
:100A8000000A0A626F6F746C6F616465722E2E2E9D
:100A90002000433E200011241FBECFEFD0E2DEBF76
:100AA000CDBF04B603FE49C08091850390918603B3
:100AB000A0918703B09188038730904BA740B04B3B
:100AC00009F03BC0109285031092860310928703B1
:100AD0001092880314BE0FB6F894A8958091600018
:100AE000886180936000109260000FBE1092010830
:100AF00010920008E3E0F0E089E080935700E49171
:100B0000E695E370E150E33040F4F0E0EE0FFF1FB4
:100B1000E35DFE4F2081318102C020E030E280E0C1
:100B200090E0A2E0B0E0821B930BA109B109B5955A
:100B3000A79597958795FC01099511E0A0E0B1E094
:100B4000ECEBFBE400E00BBF02C007900D92A43376
:100B5000B107D9F723E0A4E3B1E001C01D92A538A5
:100B6000B207E1F70E9435110C94DC250C940000CB
:100B7000FF93EF93E0913401F0913501309709F044
:100B80000995EF91FF910895FC018591803011F056
:100B9000EFDFFBCF0895FF27E0E230E247FF0CC014
:100BA000419597FF09C0EDE260957095809590950D
:100BB000611D711D811D911D27FF02C0219530E32C
:100BC00050E2AA27660F771F881F991FAA1FA41734
:100BD00010F0A41B63955A95A9F7AA3008F0A95FF5
:100BE000A05DAF93F395611571058105910541F7FE
:100BF000ED3211F4EF93F395F21718F43F93F39558
:100C0000FBCF8F91B5DFFA95E1F70895E991F9915E
:100C10008591803021F0853219F0AADFF9CF08954F
:100C200020E0E89455915532C1F3503311F46894A3
:100C300055915A3348F4505390F3220F022E220F4D
:100C4000220F200D250FF4CF0EF421958991999153
:100C5000533619F3533729F1533559F1BC0188271D
:100C60009927E8945C3621F489919991689455917B
:100C7000543639F446EF7EF077FF0DC08FEF9FEFCB
:100C80000AC055374AE039F0583540E121F0523674
:100C900042E009F00895FF93EF937DDFEF91FF911C
:100CA000B7CFFF93EF93FC0181918030B9F360DF00
:100CB000FBCFFF93EF9368DFF1CFDF93CF93CDB7F7
:100CC000DEB72596A3DFCF91DF910895282F80917D
:100CD0003F01823071F08330B1F0813001F5E62FB1
:100CE000F0E038E0739FE00DF11D1124E857FC4F50
:100CF00013C0E62FF0E088E0789FE00DF11D11248D
:100D0000E85FFC4F09C0E62FF0E038E0739FE00D8C
:100D1000F11D1124E857FD4FE491E03819F480E00B
:100D200090E008959E2F9077892F90E034E095957C
:100D300087953A95E1F738E0239F800D911D1124A6
:100D400044E0880F991F4A95E1F7EF709C012E0F40
:100D5000311DF901EE0FFF1FE050F8498591949184
:100D600008955998519A08955198599A0895589804
:100D7000509A08955098589A08955198599A85E034
:100D80008A95F1F7000089B1869581700895509891
:100D9000589A85E08A95F1F7000089B1817008952D
:100DA000CF93DF93EC010E94BD06882341F020978A
:100DB00031F085E08A95F1F700002197F4CFCE015C
:100DC000DF91CF910895CF93DF93C2E3D0E00E94EB
:100DD000BD06811108C0209731F085E08A95F1F7B2
:100DE00000002197F4CFCE01DF91CF9108952E9886
:100DF00026982F9827980E94B1060E94BA06E9E625
:100E0000F0E0808188608083E9980895E19AE99A0A
:100E10000E94B4060C94BA06E9980E94B1060C949C
:100E2000BA06CF932FB7F8948091020190910301F5
:100E3000AC01442741155F4F21F0C92FAC015F6F12
:100E400007C08F3F4FEF940741F0C82F4FEF5FEF80
:100E5000509303014093020101C0CFEF2FBF9C01CB
:100E60002F6F2F3F3F4F81F02091720320FF1FC053
:100E70009F938F938FE094E09F938F930E945D06E2
:100E80000F900F900F900F90CF3F99F080917203C9
:100E900080FF12C01F92CF9388E094E09F938F93BE
:100EA0000E945D060F900F900F900F9005C0CF3FEE
:100EB00019F48FEF9FEF02C08C2F90E0CF9108952F
:100EC000CF93CAE1C15069F00E9411078F3F2FEF05
:100ED000920749F48FE99FE00197F1F700C0000005
:100EE000F1CF8FEF9FEFCF91089580E090E890933E
:100EF0000101809300018FEF9FEF90930301809396
:100F000002010895EF92FF920F931F93CF93DF9307
:100F1000082F109237018091720380FF0CC01F923E
:100F20000F9386E194E09F938F930E945D060F904C
:100F30000F900F900F90E9980E94B1060E94BA0698
:100F40008FE891E00197F1F700C000000E94B7061A
:100F50000E94B40680E197E20E94D006892B11F42A
:100F600081E079C0C0E0D0E0FF24F39410E0EE24EB
:100F7000E39490E59A95F1F7C8010C2E02C095957F
:100F800087950A94E2F780FF04C0FE240E94BA0607
:100F900002C00E94B7060E94E306892B11F482E08A
:100FA0005AC082E390E00E94D006892B11F483E0BE
:100FB00052C02196C830D105E1F680E58A95F1F757
:100FC000FF2019F00E94BA0602C00E94B7060E94D4
:100FD000E306892B11F484E03EC082E390E00E9496
:100FE000D006892B11F485E036C090E59A95F1F78B
:100FF0000E94BA06C2E3D0E00E94C706882341F0EF
:10100000209741F025E02A95F1F700002197F4CFD1
:10101000CD2B11F486E01FC082E390E00E94D00641
:10102000892B11F487E017C00E94E306892B19F081
:10103000C2E3D0E009C088E00EC0209759F085E0F7
:101040008A95F1F7000021970E94C7068823A9F32B
:10105000CD2BB9F489E0809337018091370180610D
:10106000809337010E94B4060E94BA06E19AE99A79
:101070008FEF9FEFDF91CF911F910F91FF90EF9036
:1010800008958FEF9FEF90930301809302010E94D8
:1010900075070E94B4060E94BA06E19AE99ADF91A8
:1010A000CF911F910F91FF90EF900C9460071F92CA
:1010B0000F920FB60F9211242F933F934F935F938C
:1010C0008F939F9329B12170809173034091000108
:1010D000509101014115504819F48093360112C016
:1010E00090913601891771F09F5F891759F090E24E
:1010F000909337018093360180E090E8909301014E
:10110000809300018091000190910101969587954F
:101110009093010180930001222349F08091000106
:10112000909101019068909301018093000180915A
:1011300000019091010199278035910509F455C06E
:1011400090F48031910509F450C020F4892B09F402
:10115000A0C067C08032910509F49BC0803491051E
:1011600009F497C05EC0803A910581F040F4803860
:10117000910509F48EC080399105B9F152C0803CC7
:10118000910531F0803D910581F14BC084E613C09B
:101190008091000190910101892F9927909301017D
:1011A0008093000183E02FC0882379F025E02A9501
:1011B000F1F700008150499BF7CF07C0882349F021
:1011C00095E09A95F1F7000081504999F7CF811188
:1011D00060C08091000190910101892F992790931F
:1011E00001018093000182E00EC080910001909186
:1011F000010136E0969587953A95E1F790930101C4
:101200008093000181E080933801809100019091EA
:10121000010199278F3F9105A1F48FEF809337014A
:1012200010C080E88093370180E090E8909301013E
:101230008093000180E09FEF90930301809302016F
:1012400028C08091020190910301882781159F4F4A
:1012500019F080E48093370180910201909103019D
:10126000982F882790930301809302012091000119
:10127000309101018091020190910301822B9093A2
:1012800003018093020180E090E890930101809334
:1012900000019F918F915F914F913F912F910F90FE
:1012A0000FBE0F901F901895CF93C82F8DEE0E9400
:1012B00082078C2FCF910C948207E82FE695E69554
:1012C000E695EF70F0E0EE5BFE4F4081282F27702F
:1012D00081E090E002C0880F991F2A95E2F7242F41
:1012E00030E028233923232B11F4842B80830895A5
:1012F000E82FE695E695E695EF70F0E0EE5BFE4FA1
:101300002081382F377081E090E002C0880F991F4C
:101310003A95E2F7422F50E048235923452B19F024
:101320008095822380830895482F50E0FA013397F7
:10133000E138F10508F048C0E45BFF4F0C94D32579
:1013400087E108958FE108958CE5089580E608957A
:1013500082E6089587E2089583E508958FE208956F
:1013600089E3089587E308958FE3089587E4089556
:101370008FE4089586E508958EE508958FE6089533
:1013800080E0089585E608958EE608958FE7089534
:1013900080E3089588E3089580E4089588E408953B
:1013A00080E5089587E508958FE5089588E108951B
:1013B00088E0089580E2089580E1089589E1089524
:1013C0008DE6089588E208958F7708958FE0089557
:1013D000CF93482F50E0FA017C97E834F105A0F54F
:1013E000E353FF4F0C94D32585E53EC08AE53CC00E
:1013F0008BE53AC08CE538C08DE536C08EE534C04B
:101400008FE532C080E630C081E62EC082E62CC077
:1014100083E62AC08FE628C081E726C082E724C081
:1014200084E722C085E720C087E71EC088E71CC08C
:101430008AE71AC08CE718C08FE716C080E714C08F
:1014400089E712C08BE710C0C82F1F928F9389EADB
:1014500094E09F938F930E945D060F900F900F90E2
:101460000F908C2F01C084E5CF9108950F931F93A7
:10147000CF93DF930E94B0238C010E941107EC01EF
:10148000019631F4C8010E94C823843F9140A8F31B
:10149000CE01DF91CF911F910F9108950E94F70621
:1014A0000C94060780917203816080937203E2E4DA
:1014B000F1E0119281E0E235F807D9F70895E82FBD
:1014C000F0E0EE5BFE4F80810895E2E4F1E01192DE
:1014D00081E0E235F807D9F70895982F80913F0110
:1014E000823049F492FB882780F990FD826091FD5B
:1014F00084600C9454090895CF93DF938091370151
:10150000882311F1809137011F928F938AE295E031
:101510009F938F930E945D068091370180750F9095
:101520000F900F900F9071F480913E01893051F42B
:1015300084E295E09F938F930E945D0610923E0196
:101540000F900F9010923701E0913E018E2F90E0A6
:101550008A30910508F0C9C3FC01EB5EFE4F0C9484
:10156000D3250E94B0239F938F938FE195E09F93A3
:101570008F930E945D0610923F01109241011092DC
:1015800040010E94650A0E94491981E035C00E940D
:101590000C072E98269A2F98279A0E94B023909392
:1015A0003D0180933C0182E00BC080913C01909111
:1015B0003D010E94C823853F914008F496C383E013
:1015C00080933E0192C32E9826982F9827980E94C8
:1015D00075070E9406070E94B0239F938F938AE1AC
:1015E00095E09F938F930E945D060E94B023909395
:1015F0003D0180933C0184E080933E010F900F9069
:101600000F900F9072C30E941107019609F46DC3E9
:101610000E94B0239F938F9385E195E09F938F93D2
:101620000E945D060E94B02390933D0180933C018F
:1016300085E0E2CF80913C0190913D010E94C8235A
:10164000853F914018F087E080933E010E9411078A
:10165000019609F44AC30E94B0239F938F9380E1BF
:1016600095E09F938F930E945D060E94B023909314
:101670003D0180933C0186E0BFCF80913C01909179
:101680003D010E94C823853F914018F087E0809378
:101690003E010E941107019609F427C30E94B0235E
:1016A0009F938F938BE095E09F938F930E945D06AD
:1016B00087E0A2CF0E94B0239F938F9386E095E0AE
:1016C0009F938F930E945D0682EF0E9482070F9086
:1016D0000F900F900F908F3F2FEF920789F08A3F66
:1016E000910589F40E94360A8F3F3FEF930771F00E
:1016F000D82FCC270E94360A9E01282BC90108C08A
:101700008FEF9FEF05C08EEF9FEF02C080E090E06B
:10171000909341018093400180913701882381F0AB
:10172000809137011F928F938BEF94E09F938F935B
:101730000E945D06109237010F900F900F900F904E
:1017400080914001909141019C01222721154BEA93
:10175000340711F482E00CC021153F4B11F483E0F3
:1017600007C00097B9F38F3F2FEF920721F481E074
:1017700080933F010DC08F3F910561F785EE94E0A6
:101780009F938F930E945D0610923F010F900F90E0
:1017900080913F011F928F93809141018F9380919F
:1017A00040018F9388ED94E09F938F930E945D0694
:1017B00088E080933E010F900F900F900F900F9054
:1017C0000F9093C20E94B0239F938F9383ED94E078
:1017D0009F938F930E945D060F900F900F900F9034
:1017E00080913F01823031F0833041F488EF0E94D4
:1017F000820704C00E94C1160E946D0A89E080938E
:101800003E010E94B0239F938F938EEC94E09F93B0
:101810008F930E945D060F900F900F900F90C091D4
:101820003F01C23009F47EC0C33009F4E3C1C130C6
:1018300009F05BC20E9411078F3F3FEF930709F445
:1018400054C29C012F7733272236310548F083ECB0
:1018500094E09F938F930E945D0610923B0141C2DA
:1018600020913B01223009F444C028F4222351F096
:10187000213019F154C0233009F447C0243009F451
:1018800049C04DC0803E910569F01CF4009739F0C5
:101890000EC0813E910549F08F3F910541F488EBE0
:1018A00094E01BC2C0933B0120C282E02BC0803871
:1018B000910508F4D5C18F770BC28633910579F174
:1018C00024F48A32910539F42AC08A3A910539F113
:1018D000863B910521F18038910528F40E94E809A2
:1018E0000E945D091CC08F770E94E8090E94780958
:1018F00016C08D31910529F08D39910581F484E070
:1019000001C083E080933B01F0C18534910539F437
:1019100085E5A6C18534910511F485E5D9C11092FC
:101920003B01E3C10E9411078F3F4FEF940709F479
:10193000DCC1E0913A014E2F50E04B30510508F0E8
:1019400056C1FA01E15EFE4F0C94D3258E35910508
:1019500009F472C07CF58732910509F46BC0ACF4D0
:101960008731910509F46AC034F4009709F068C022
:101970008EE994E063C18931910509F46CC18F311E
:10198000910509F05DC08FE16BC18933910509F4C0
:101990004DC034F48F32910509F052C087E560C123
:1019A0008335910509F444C08C35910509F048C090
:1019B00089E156C18A3A910509F495C18CF48038C1
:1019C000910591F12CF48F369105D1F58CE548C144
:1019D0008338910539F18438910591F58FE6EAC095
:1019E000803F9105E9F044F4803E9105B9F0813ED5
:1019F000910531F584E0E1C08C3F910509F473C194
:101A00008F3F9105E9F40E94650A83E994E09F9372
:101A10008F930E945D0610923A0163C182E0CDC0AF
:101A200081E0CBC082E0C6C089E0C7C08EE618C1A5
:101A300085E616C187E614C184E612C187E710C1A6
:101A40008038910508F40CC10E94650A87E894E08B
:101A500044C18935910509F4CAC0803F910521F040
:101A60008231910519F4C3C083E0A7C010923A01F6
:101A70008038910518F40E949409F2C00E94650A0A
:101A80008DE794E02AC18933910581F1A4F48F3167
:101A9000910581F144F48731910591F189319105E6
:101AA00089F58FE7A2C08732910531F18F32910518
:101AB00049F587E59AC08E35910501F144F48335E7
:101AC0009105B1F08C359105E9F489E18EC0833838
:101AD000910541F08438910539F08F36910591F4E4
:101AE0008CE583C082E081C08FE67FC08EE67DC03A
:101AF00085E67BC08FE179C087E677C084E675C054
:101B000087E773C010923A018038910508F4E0C06D
:101B10000E94650A83E794E0E0C010923A018231A6
:101B2000910509F4E2C08935910509F4DEC08038D9
:101B3000910518F40E949409CBC00E94650A86E6BC
:101B400094E0CBC08431910531F0803F910509F0DC
:101B50004EC086E032C085E030C08737910509F07D
:101B600046C080E027C0449709F041C087E025C007
:101B7000803F9105E1F588E020C087379105B9F5F0
:101B800080E033C08532910591F03CF486319105B7
:101B900081F04E97A9F483E10DC08632910529F0BA
:101BA000803F910569F48AE008C08AE603C088E6B0
:101BB00001C081E50E945D091AC080933A0195C079
:101BC0000E94650A14C08E31910571F024F4469785
:101BD000B9F781E50AC08532910521F0869781F732
:101BE0008AE603C088E601C083E10E94780910926A
:101BF0003A017BC00E9411078F3F2FEF920709F433
:101C000074C020913901222319F0213079F16DC07F
:101C10008438910501F13CF4009771F08338910507
:101C2000E1F482E01DC0803F910589F08F3F91056E
:101C3000A1F480E594E051C08BE594E09F938F93ED
:101C40000E945D060E94650A0E94491931C081E028
:101C5000809339014AC08FE703C08038910518F49A
:101C60000E945D0942C083E494E037C08338910547
:101C700011F17CF4009739F585E394E09F938F93FD
:101C80000E945D060E94650A0E944919109239015E
:101C90000FC08438910589F08F3F9105A1F487E248
:101CA00094E09F938F930E945D061092390119C0B2
:101CB0000F900F901AC082E001C08FE70E94780950
:101CC0001092390112C0109239018038910518F430
:101CD0000E9478090AC08DE194E09F938F930E943F
:101CE0005D060F900F9010923E0181E0DF91CF9141
:101CF00008958091760208950895CF93DF9300D0E0
:101D00001F92CDB7DEB720917C03243021F523E06C
:101D100029839B838A8382E08093E9008FEF9091EF
:101D2000E800815095FD06C095ED9A95F1F7000009
:101D30008111F5CF8091E80085FF0DC040E050E0B3
:101D400063E070E0CE0101960E94E9128091E80004
:101D50008E778093E8000F900F900F90DF91CF91D6
:101D60000895CF93DF9300D01F92CDB7DEB72091B7
:101D70007C03243029F522E02983805891099B8334
:101D80008A832093E9008FEF9091E800815095FDC0
:101D900006C095ED9A95F1F700008111F5CF80917D
:101DA000E80085FF0DC040E050E063E070E0CE0148
:101DB00001960E94E9128091E8008E778093E800F6
:101DC0000F900F900F90DF91CF910895CF93DF93F5
:101DD000EC0190917C03943009F048C0809114018B
:101DE0008823D9F0809115018823B9F09093E900F8
:101DF00081E8815049F09091E80095FD05C09AE294
:101E00009A95F1F700C0F5CF8091E80085FF2EC0CC
:101E100040E050E060E270E019C081E08093E900AA
:101E200081E8815059F09091E80095FD07C0EFE3FB
:101E3000F1E03197F1F700C00000F3CF8091E800A6
:101E400085FF14C040E050E068E070E0CE010E94E1
:101E5000E9128091E8008E778093E80080E2FE012D
:101E6000A6E5B2E001900D928A95E1F7DF91CF915E
:101E70000895CF93C0915401C1110BC00E94BC239F
:101E8000643C79408105910520F081E08093540104
:101E9000C1E08C2FCF910895FF920F931F93CF93A2
:101EA000DF93D82F0FB607FE83C080917C03843068
:101EB00081F08091070190E001962091090130E0C6
:101EC000822393232091080130E08217930709F0C1
:101ED000CBC00E94390F811110C08091070190E0A2
:101EE00001962091090130E082239323209108017B
:101EF00030E08217930709F0B7C00E94B0238C012D
:101F0000C091E900CF709091EC00892F817090FD15
:101F100080E8C82B83E08093E90085E0F82E80916B
:101F2000EB0085FD42C08091EB0080FF3EC08091B8
:101F3000EE0087FF3AC08091080190910701981741
:101F400009F457C09091E80095FF8CC0E09105011D
:101F5000F0910601E80FF11D20818F5F909109013A
:101F60008923809308012093F1008091E80085FD8A
:101F7000E2CF8091E80080FFDECF8091E8008E778D
:101F80008093E800F0920401D6CF8091070190E0A1
:101F900001962091090130E08223932320910801CA
:101FA00030E08217930709F44AC0CF70C093E9006C
:101FB00040910701842F90E001962091090130E0C3
:101FC000822393232091080130E08217930709F4BC
:101FD0004EC0E0910501F0910601E40FF11DD083A0
:101FE000809107018F5F90910901892380930701F8
:101FF0003EC08091E80085FF35C0D093F10081E0BC
:102000002091F2003091F300232B91F09091E800A1
:1020100090FF0EC09091E80095FF03C01092F10070
:10202000F9CF9091E8009E779093E800F092040138
:10203000882309F4AACFCF70C093E90018C080911B
:102040000401882309F4B1CF0E94B0239C018017BA
:10205000910711F4890163CF9091040191509093FD
:102060000401F8CF80E0CCCF40910701B2CF80E0EF
:10207000DF91CF911F910F91FF90089580917B0385
:10208000811104C00E9451150C94B315089510924B
:102090007B030895089542E061EC81E00E946212A2
:1020A00042E061EC82E00E94621242E261EC83E075
:1020B0000E94621242E261EC84E00C946212809110
:1020C0007E03833009F455C030F4813071F08230E2
:1020D00009F48EC008958A3009F47AC08B3009F46F
:1020E00060C0893009F09CC020C080917D03813A96
:1020F00009F096C08091E800877F8093E800809186
:10210000810390918203892B21F460E286E592E0BD
:1021100003C060E080E090E070E00E9436138091A0
:10212000E8008B778093E800089580917D038132E9
:1021300009F076C08091810390918203009719F095
:10214000039709F06DC08091E800877F8093E800D5
:102150008091E80082FD05C080917C038111F8CF59
:102160005FC08091F100809376028091E8008B77C8
:1021700053C080917D03813A09F052C08091810360
:1021800090918203892B09F04BC08091E800877FF2
:102190008093E8008091E80080FFFCCF80911401DB
:1021A00036C080917D038132D9F580918103909171
:1021B0008203892BA9F58091E800877F8093E8004E
:1021C0000E94971280917F03809314010C94491907
:1021D00080917D03813221F58091E800877F809393
:1021E000E8000E94971280918003809377020895FF
:1021F00080917D03813AA1F48091E800877F8093EC
:10220000E8008091E80080FFFCCF80917702809306
:10221000F1008091E8008E778093E8000C9497128B
:1022200008958091760280935501109276020E9463
:10223000650A0C9449190C9411110E945D23809138
:102240007A03882329F00E946A2381110C944C128E
:1022500008950E947E23809155018093760208950F
:102260000C94291108950C943211CF9384B7877F71
:1022700084BF0FB6F894A895809160008861809320
:102280006000109260000FBE90E080E80FB6F894F6
:1022900080936100909361000FBE8CE49FE00E94E8
:1022A00030238AE091E00E94BC1689E595E00E9407
:1022B000C4050E944E0A0E9470170E9451150E9488
:1022C000B31578940E94721780917C03843029F0B2
:1022D0000E94A1160E943211F7CF87E495E00E9478
:1022E000C4050E94331185E395E00E94C405C3E054
:1022F00080917C03853019F40E941D11F9CF0E9452
:1023000076172091E4003091E50080915201909180
:1023100053012817390709F466C08091E4009091B1
:10232000E50090935301809352010E94390F882356
:1023300009F459C080917C03843009F054C0809125
:10234000E9008F702091EC00922F917020FD90E8B1
:10235000892BC093E9009091EB0090FF41C09091D0
:10236000EE0097FF3DC090910801209107012917C9
:1023700009F12091E80025FF1DC0E0910501F091D1
:102380000601E90FF11D30819F5F20910901922321
:10239000909308013093F1009091E80095FDE3CF10
:1023A0009091E80090FFDFCF9091E8009E779093A6
:1023B000E800D9CF2091F2003091F300232B81F077
:1023C0009091E80090FF0CC09091E80095FF03C049
:1023D0001092F100F9CF9091E8009E779093E80079
:1023E0008F708093E9000E94A11682CF292F332796
:1023F00023303105C9F060F42130310581F02230FD
:10240000310509F041C084E790E029EB35E040C098
:1024100021323105E1F02232310531F135C082E15E
:1024200090E02DE236E034C099278130910549F0E3
:1024300028F0029749F5EFE6F5E005C0E5EBF5E099
:1024400002C0E5EAF5E0849190E09F0121C064308C
:102450007105D0F4660F771FFB01EC5DFE4F208104
:10246000318189E090E014C06430710568F4FB01AB
:10247000EE0FFF1FE45EFE4F20813181FB01E85E1D
:10248000FE4F808190E004C080E090E020E030E0EA
:10249000FA0131832083089584E189BD86E189BDF5
:1024A00009B400FEFDCF8091D8008F7D8093D800C5
:1024B0008091E00082608093E0008091E00081FDE7
:1024C000FCCF0895982F973068F59093E9009817FE
:1024D00039F07091EC002091ED005091F00003C0B4
:1024E000242F762F50E021FD02C09F5FECCF30916A
:1024F000EB003E7F3093EB003091ED003D7F309359
:10250000ED003091EB0031603093EB007093EC0004
:102510002093ED005093F0002091EE0027FDE5CFD1
:1025200080E008958F708093E90081E008958091A4
:102530007D0387FF11C08091E80082FD05C0809176
:102540007C038111F8CF11C08091E8008B770BC01C
:1025500080917C03882349F08091E80080FFF8CFC8
:102560008091E8008E778093E80008952091E40040
:102570003091E50095E64091EC00842F817040FF9A
:1025800023C08091E80080FD1DC080917C038823DA
:1025900099F0853099F08091EB0085FD11C0409154
:1025A000E4005091E5002417350729F3915011F00C
:1025B0009A01E1CF84E0089582E0089583E00895D0
:1025C00081E0089580E008954091E80042FFDDCF6A
:1025D0000895CF92DF92EF92FF920F931F93CF93C4
:1025E000DF93EC018B017A010E94B612811135C094
:1025F000E114F10439F0F70180819181081B190B76
:10260000C80FD91FC12CD12C0115110529F18091BA
:10261000E80085FD18C08091E8008E778093E8007F
:102620000E94A116E114F10449F0F7018081918123
:10263000C80ED91ED182C08285E00FC00E94B6129A
:10264000882311F30AC089918093F1000150110988
:10265000FFEFCF1ADF0AD8CF80E0DF91CF911F9133
:102660000F91FF90EF90DF90CF900895209183031A
:10267000309184032617370748F06115710539F446
:102680002091E8002E772093E80001C0B901FC01F9
:1026900020E06115710569F180917C038823E1F1E7
:1026A0008530E1F18091E80083FD3AC08091E80037
:1026B00082FD2CC08091E80080FFEBCF8091F2007A
:1026C0009091F3006115710551F08830910538F44F
:1026D00021912093F100615071090196F3CF21E01F
:1026E000089709F020E08091E8008E778093E80059
:1026F000D0CF2111D1CF0AC080917C03882361F013
:10270000853061F08091E80083FD0AC08091E80087
:1027100082FFF2CF80E0089582E0089583E008957B
:1027200081E00895209183033091840326173707B1
:1027300048F06115710539F42091E8002E77209357
:10274000E80001C0B901FC0120E06115710581F1CB
:1027500080917C03882309F43EC0853009F43DC094
:102760008091E80083FD3BC08091E80082FD2DC090
:102770008091E80080FFE9CF8091F2009091F30012
:102780006115710559F08830910540F4249120932A
:10279000F1003196615071090196F2CF21E008975E
:1027A00009F020E08091E8008E778093E800CDCF9B
:1027B0002111CECF0AC080917C03882361F085303F
:1027C00061F08091E80083FD0AC08091E80082FFFB
:1027D000F2CF80E0089582E0089583E0089581E0DB
:1027E00008951F93CF93DF93CDB7DEB7AA970FB6A7
:1027F000F894DEBF0FBECDBFEDE7F3E08091F100AE
:10280000819323E0E538F207C9F70E945F108091B9
:10281000E80083FF2EC180917D0390917E03492FB4
:1028200050E04A30510508F024C1FA01E65DFE4F40
:102830000C94D325803821F0823809F01AC108C0E1
:102840008091790390917A03992389F082600FC077
:10285000809181038F70873008F00BC18093E9006D
:102860008091EB0085FB882780F91092E900909118
:10287000E800977F9093E8008093F1001092F100B8
:10288000D1C0282F2D7F09F0F4C0882319F08230A1
:1028900061F0EFC080917F03813009F0EAC093308E
:1028A00009F080E080937A032EC080917F0381112C
:1028B0002AC0809181038F702FEF280F263008F0F7
:1028C000D8C08093E9002091EB0020FF1CC093301A
:1028D00021F48091EB00806214C09091EB00906134
:1028E0009093EB0021E030E0A90102C0440F551F96
:1028F0008A95E2F74093EA001092EA008091EB009B
:1029000088608093EB001092E9008091E800877F57
:102910008093E8000E949712ACC08111AAC0109168
:102920007F031F778091E3008078812B8093E30001
:102930008091E800877F8093E8000E949712809141
:10294000E80080FFFCCF8091E30080688093E30083
:10295000111102C082E001C083E080937C0389C032
:102960008058823008F085C080917F039091800369
:102970008C3D53E0950779F583E08A838AE2898369
:102980004FB7F894DE01139620E03EE051E2E32FCA
:10299000F0E050935700E49120FF03C0E295EF7000
:1029A0003F5FEF708E2F90E0EA3010F0C79601C0C5
:1029B000C0968D939D932F5F243149F74FBF80912F
:1029C000E800877F8093E8006AE270E0CE0101961C
:1029D0000E94361316C06091810370918203AE018C
:1029E0004F5F5F4F0E94F611BC01892B09F441C073
:1029F0009091E800977F9093E80089819A810E94E6
:102A000092138091E8008B778093E80032C0803881
:102A100081F58091E800877F8093E80080917803BA
:102A20008093F1008091E8008E7772CF811121C0F0
:102A300080917F039091800399270297D4F480912D
:102A4000E800877F8093E80080917F03809378037C
:102A50000E94971280917803811106C08091E30053
:102A600087FD02C081E001C084E080937C030E9466
:102A70004B108091E80083FF0AC08091E800877FB7
:102A80008093E8008091EB0080628093EB00AA962F
:102A90000FB6F894DEBF0FBECDBFDF91CF911F916F
:102AA00008950E94C2150E94CA15E0EEF0E08081F0
:102AB00081608083E8EDF0E080818F77808319BCAE
:102AC000A7EDB0E08C918E7F8C9380818F7E808388
:102AD00010927B0308950F931F93CF93DF930E946F
:102AE000C2150E94CA15C8EDD0E088818F7788830F
:102AF00088818068888388818F7D8883E7EDF0E016
:102B000080818068808319BC10927C0310927803C6
:102B100010927A031092790300EE10E0F8018081A0
:102B20008B7F808388818160888342E060E080E0E1
:102B30000E946212E1EEF0E080818E7F8083E2EEFF
:102B4000F0E0808181608083808188608083F801EB
:102B500080818E7F8083888180618883DF91CF919F
:102B60001F910F910895E8EDF0E080818F7E8083C2
:102B7000E7EDF0E080818160808381E080937B03DA
:102B80000C946B15E8EDF0E080818C7F80831092CF
:102B9000E20008951092DA001092E10008951F9269
:102BA0000F920FB60F9211240BB60F922F933F93F3
:102BB0004F935F936F937F938F939F93AF93BF9345
:102BC000EF93FF938091E10082FF0BC08091E200C0
:102BD00082FF07C08091E1008B7F8093E1000E941B
:102BE000A0168091DA0080FF1FC08091D80080FF7E
:102BF0001BC08091DA008E7F8093DA008091D9002B
:102C000080FF0DC084E189BD86E189BD09B400FE65
:102C1000FDCF81E080937C030E943E1005C019BC6B
:102C200010927C030E9447108091E10080FF19C040
:102C30008091E20080FF15C08091E2008E7F80933A
:102C4000E2008091E20080618093E2008091D800F0
:102C500080628093D80019BC85E080937C030E9439
:102C60001B118091E10084FF30C08091E20084FF5D
:102C70002CC084E189BD86E189BD09B400FEFDCF89
:102C80008091D8008F7D8093D8008091E1008F7E65
:102C90008093E1008091E2008F7E8093E20080913A
:102CA000E20081608093E20080917803882311F034
:102CB00084E007C08091E30087FD02C081E001C08D
:102CC00083E080937C030E9430118091E10083FFB8
:102CD00024C08091E20083FF20C08091E100877FC3
:102CE0008093E10082E080937C03109278038091CE
:102CF000E1008E7F8093E1008091E2008E7F8093DF
:102D0000E2008091E20080618093E20042E060E0B6
:102D100080E00E9462120E944A10FF91EF91BF91E1
:102D2000AF919F918F917F916F915F914F913F9163
:102D30002F910F900BBE0F900FBE0F901F90189504
:102D40000895CF9380917C038823A1F0C091E9007E
:102D5000CF709091EC00892F817090FD80E8C82B96
:102D60001092E9008091E80083FD0E94F113CF707A
:102D7000C093E900CF91089590937D0280937C02E7
:102D80000895E0917C02F0917D02309721F001904E
:102D9000F081E02D099480E00895EF92FF920F9367
:102DA0001F93CF93DF93E0917C02F0917D023097E7
:102DB000B1F18C010280F381E02D099580917203BD
:102DC00082FF2DC080FF04C086E397E00E94C40507
:102DD000E80110E280E3E82E87E0F82E809172038C
:102DE00080FF0BC088811F928F93FF92EF920E9409
:102DF0005D060F900F900F900F90115021961111BA
:102E0000EDCF8091720380FF0AC08EE297E0DF91E0
:102E1000CF911F910F91FF90EF900C94C405DF911B
:102E2000CF911F910F91FF90EF900895CF93DF9373
:102E300020917A0230917B022817390709F190938B
:102E40007B0280937A02E0917C02F0917D023097C0
:102E5000B9F0EC010680F781E02D099580917203AD
:102E600082FF0EC080FF0CC0DF93CF9380E297E01B
:102E70009F938F930E945D060F900F900F900F907D
:102E8000DF91CF910895CF93DF9320917802309115
:102E900079022817390709F1909379028093780213
:102EA000E0917C02F0917D023097B9F0EC01008452
:102EB000F185E02D09958091720382FF0EC080FF9D
:102EC0000CC0DF93CF9380E197E09F938F930E9494
:102ED0005D060F900F900F900F90DF91CF910895A6
:102EE0000C9419180E94A7230C94520ABF92CF92F7
:102EF000DF92EF92FF920F931F93CF93DF9300D057
:102F000000D01F92CDB7DEB70E947C0A0FE712E017
:102F1000F12C8F2D0E945F0AB82EF801C080C826C0
:102F200039F4F3940F5F1F4FF0E1FF12F2CF30C07E
:102F30008091720381FD0E941A18D12CEE24E39433
:102F40008C2D8E21F9F0D982FA8291E08B2D8E2181
:102F500009F490E09B830E94B0238160782F9D83C9
:102F60008C8349815A816B818D810E9450184981DF
:102F70005A816B817C818D810E944823F801808178
:102F80008E258083D394EE0CF8E0DF12D9CFC9CF21
:102F90008FEF89838A831B820E94B0238160782F00
:102FA0009D838C8349815A816B818D810E94501849
:102FB0000E9447230E94C11690917E02891741F119
:102FC0000E94C11680937E029091720392FF0EC000
:102FD00090FF0CC01F928F9381E497E09F938F9393
:102FE0000E945D060F900F900F900F9080917E02CF
:102FF0000F900F900F900F900F90DF91CF911F9136
:103000000F91FF90EF90DF90CF90BF900C945923D9
:103010000F900F900F900F900F90DF91CF911F9115
:103020000F91FF90EF90DF90CF90BF9008950C9498
:103030006D0A0895EF92FF920F931F93CF93DF9342
:103040008AE597E00E94C405C0E0D0E08CE2E82E5B
:1030500081E0F82E0CE417E08C2F0E945F0A0E949A
:103060003523FF92EF921F928F93DF93CF931F939D
:103070000F930E945D0621968DB79EB708960FB6F6
:10308000F8949EBF0FBE8DBFC031D10529F7DF91E7
:10309000CF911F910F91FF90EF900895089508959B
:1030A000CF93DF93CDB7DEB72B970FB6F894DEBF83
:1030B0000FBECDBF942F4F83252F588769877A87FE
:1030C0008B874A855B85452B31F02F3F31F481E0BA
:1030D0009F3F19F403C081E001C080E080FD07C07C
:1030E0004F81588569857A858B850E944823DE014A
:1030F000119686E0FD0111928A95E9F785E0FE01BF
:10310000379601900D928A95E1F749815A816B813A
:103110007C818D819E810E94431F2B960FB6F8946F
:10312000DEBF0FBECDBFDF91CF910895CF9388232F
:1031300009F465C0C82F8CEF8C0F813A20F080E530
:103140008C0F8E3248F48C2F0E948025811157C03D
:103150008C2F0E942B220CC080E28C0F883058F4F8
:10316000C77081E001C0880FCA95EAF70E94D0229B
:10317000CF910C940A238BE58C0F833078F4C53AF9
:1031800029F0C63A31F083E890E005C081E890E08C
:1031900002C082E890E0CF910C94161788E58C0F5E
:1031A000853168F5C83A89F0C93A91F0CA3A99F080
:1031B000CB3AA1F0CC3AA9F0CD3AB1F0CE3AB9F081
:1031C000CF3AC1F080E090E017C082EE90E014C0EA
:1031D00089EE90E011C08AEE90E00EC085EB90E0A1
:1031E0000BC086EB90E008C083EB90E005C084EB59
:1031F00090E002C087EB90E0CF910C944317CF9101
:103200000895882349F19CEF980F913A20F090E5BA
:10321000980F9E3218F40E947B220DC090E2980F06
:10322000983058F4877091E001C0990F8A95EAF7B9
:10323000892F0E94D6220C940A239BE5980F933085
:1032400020F480E090E00C941617885A853120F421
:1032500080E090E00C9443170895882321F00E94A9
:10326000D0220C940A230895882321F00E94D622AC
:103270000C940A2308950E94F0220E94BF220E940B
:103280000A2380E090E00E94161780E090E00C9402
:1032900043170E94E0220C943B19CF92DF92EF92E9
:1032A000FF920F931F93CF93DF9300D000D01F9214
:1032B000CDB7DEB76C010E945B238111EAC285E0C5
:1032C000F601DE01119601900D928A95E1F7F60163
:1032D00040815181238134812115310531F05F3FD7
:1032E00031F481E04F3F19F403C081E001C080E078
:1032F00080FDCFC2F601F280E580E2948FE0E82203
:1033000049835A83FB82722F3D832C836F2D8D81DD
:103310000E94A7218C010E94A6210E949620E12FE5
:10332000E295EF708E2F90E0FC01EC5CFE4F0C9468
:10333000D325812F807F1F70882311F01295107F75
:10334000FF2049F0112309F43BC2812F0E94E322A0
:103350000E940A2335C2802F0E940119112309F40B
:1033600098C2812F0E94E9220F900F900F900F902A
:103370000F90DF91CF911F910F91FF90EF90DF9011
:10338000CF900C940A23812F807F1F70803211F020
:103390001295107F002319F0013009F12BC0FF2096
:1033A000A9F0EE2059F1F1E0812FEF1228C00F9023
:1033B0000F900F900F900F90DF91CF911F910F9171
:1033C000FF90EF90DF90CF900C94F322EE2021F04D
:1033D00021E0E21609F45DC20E94F6222DC0FF2012
:1033E000E9F085E08E1508F454C20E94CD228123B5
:1033F00029F022C0FF20F1F0E11015C0812F0F90BD
:103400000F900F900F900F90DF91CF911F910F9120
:10341000FF90EF90DF90CF900C942D1994E09E15C3
:1034200008F437C209C0F601858180FFC9C18F70D9
:103430008583E4CFE110D7C1812F4AC1812F8695C2
:103440008695837019F08130B9F023C2FF2019F0FE
:10345000C801937002C080E090E00F900F900F9031
:103460000F900F90DF91CF911F910F91FF90EF90F0
:10347000DF90CF900C941617FF2019F0C8019370BD
:1034800002C080E090E00F900F900F900F900F908F
:10349000DF91CF911F910F91FF90EF90DF90CF9030
:1034A0000C944317812F837009F070C0F110F1C1A3
:1034B000202F229526952770220F220F602F6F70E4
:1034C000862F90E0A0E0B0E06C017D01022E04C0E8
:1034D000CC0CDD1CEE1CFF1C0A94D2F704FF12C0BA
:1034E0008FE090E0A0E0B0E004C0880F991FAA1F11
:1034F000BB1F2A95D2F7BC01CD01609570958095D0
:10350000909503C060E070E0CB011695169513709E
:103510001230B1F040F56C297D298E299F29113098
:1035200031F10F900F900F900F900F90DF91CF918E
:103530001F910F91FF90EF90DF90CF900C94BB20E4
:103540006C297D298E299F290F900F900F900F9045
:103550000F90DF91CF911F910F91FF90EF90DF902F
:10356000CF900C94D5200E94BB20C701B6010F90CC
:103570000F900F900F900F90DF91CF911F910F91AF
:10358000FF90EF90DF90CF900C94A120FF2019F0D6
:10359000812F817001C08695882309F47AC1202F7C
:1035A000229526952770220F220F602F6F70862F8D
:1035B00090E0A0E0B0E06C017D01022E04C0CC0CD4
:1035C000DD1CEE1CFF1C0A94D2F704FF12C08FE032
:1035D00090E0A0E0B0E004C0880F991FAA1FBB1FB5
:1035E0002A95D2F7BC01CD01609570958095909594
:1035F00003C060E070E0CB01169516951370123091
:10360000B1F040F56C297D298E299F29113031F1C7
:103610000F900F900F900F900F90DF91CF911F910F
:103620000F91FF90EF90DF90CF900C9482216C2946
:103630007D298E299F290F900F900F900F900F904A
:10364000DF91CF911F910F91FF90EF90DF90CF907E
:103650000C9494210E948221C701B6010F900F9013
:103660000F900F900F90DF91CF911F910F91FF90CE
:10367000EF90DF90CF900C947021003FC1F128F4BF
:1036800080E4800F803250F096C0023F09F45EC0A3
:1036900008F449C0033F09F46CC08DC0F02FF071ED
:1036A000EF2E812F8F71FF2051F00E940921802F72
:1036B000EE2019F08295807FA2CE8F70A0CE0E945E
:1036C0002A21802FEE2019F08295807F01C08F7013
:1036D0000F900F900F900F900F90DF91CF911F914F
:1036E0000F91FF90EF90DF90CF900C943419FF2052
:1036F000A9F024E02E1508F4CCC0812F8F710F9013
:103700000F900F900F900F90DF91CF911F910F911D
:10371000FF90EF90DF90CF900C944F2185E08E15B5
:1037200008F4B7C0EACFFF2099F0812F8F710F9076
:103730000F900F900F900F90DF91CF911F910F91ED
:10374000FF90EF90DF90CF900C940921FF2069F358
:10375000812F8F710F900F900F900F900F90DF912E
:10376000CF911F910F91FF90EF90DF90CF900C942D
:103770002A21FF2089F0812F8F710F900F900F90D9
:103780000F900F90DF91CF911F910F91FF90EF90CD
:10379000DF90CF900C94F4200F900F900F900F902B
:1037A0000F90DF91CF911F910F91FF90EF90DF90DD
:1037B000CF900C94EF20FF2099F0EE2009F4B5CFC4
:1037C000802F0F900F900F900F900F90DF91CF915F
:1037D0001F910F91FF90EF90DF90CF900C9496186F
:1037E000EE2009F4B5CF802F0F900F900F900F901F
:1037F0000F90DF91CF911F910F91FF90EF90DF908D
:10380000CF900C940119412F4F70602FC6010E9478
:103810001B240F900F900F900F900F90DF91CF917E
:103820001F910F91FF90EF90DF90CF900C94F11FBC
:1038300001112FC0FF2069F10E9449199FEFE0E7B5
:10384000F2E09150E040F040E1F700C000000F903E
:103850000F900F900F900F90DF91CF911F910F91CC
:10386000FF90EF90DF90CF900C94FC23412F4F708E
:10387000602FC6010F900F900F900F900F90DF9167
:10388000CF911F910F91FF90EF90DF90CF900C940C
:103890001E240F900F900F900F900F90DF91CF91FB
:1038A0001F910F91FF90EF90DF90CF9008951F939D
:1038B000CF93DF9300D000D01F92CDB7DEB7942F07
:1038C0004983252F5A836B837C838D834C815D8153
:1038D000452B31F02F3F31F481E09F3F19F403C0B5
:1038E00081E001C080E0182F117080FD31C0498156
:1038F0005A816B817C818D810E94A721292F22957D
:103900002F702C3030F42A30A0F42250223030F0C6
:1039100022C02C30C9F02F30B9F01DC0853A28F4F0
:103920008430C0F4823028F415C090E2980F9830AB
:1039300088F0883E30F4803E68F48450813A58F430
:1039400009C0803F41F406C093FB112710F903C062
:1039500010E001C011E0812F0F900F900F900F9099
:103960000F90DF91CF911F910895CF93DF9300D0F7
:1039700000D01F92CDB7DEB70F900F900F900F9031
:103980000F90DF91CF910895CF93DF9300D000D0B7
:1039900000D0CDB7DEB726960FB6F894DEBF0FBEC7
:1039A000CDBFDF91CF9108951F93CF93DF93C09147
:1039B0008F0216E080919002C81799F0D0E01C9F0A
:1039C000F0011D9FF00D1124EF56FD4F40815181F4
:1039D00062817381848195810E94C41C2196C77085
:1039E000E9CFDF91CF911F9108954091C10250918D
:1039F000C2026091C3027091C4028091C50290918D
:103A0000C6020C94C41C0F931F93CF93DF93809135
:103A1000C60282958F7009F05DC08091C302882331
:103A200009F458C080918F02109190026091C102F8
:103A30007091C202C091C402D091C50291E06F3F63
:103A400009F090E0292F06E0811709F443C0209780
:103A500021F07F3F21F030E003C031E001C0322F80
:103A600090E030FD34C0089FF001099FF00D112453
:103A7000DF01AF56BD4F11963C911197371327C008
:103A80003C91361324C012963C91129731111FC0FD
:103A900013964D915C9114974C1B5D0B483C51055E
:103AA000B0F48091C6028F7080618093C602EA569E
:103AB000FD4F80818F708061808381EC92E00E9455
:103AC0004D19DF91CF911F910F910C94D41C019649
:103AD0008770BACFDF91CF911F910F9108959F9278
:103AE000AF92BF92CF92DF92EF92FF920F931F930C
:103AF000CF93DF93CDB7DEB761970FB6F894DEBFF3
:103B00000FBECDBF8C0185E0F801DE011D9601904E
:103B10000D928A95E1F7F80140815181F280C380CE
:103B2000D4809091C1026091C2022091C402309170
:103B3000C5022115310531F06F3F31F481E09F3F1F
:103B400019F403C081E001C080E0F82FF1709F2ECE
:103B500080FD52C181ECA82E82E0B82EE090C30215
:103B6000F601E21BF30BEE2009F4E8C08091C602D7
:103B7000E83CF10508F0A4C0282F207F09F053C0CD
:103B8000561313C0491311C0EF2CF1100EC08F70E3
:103B900080618093C6020E94F51CC5010E944D19E8
:103BA0008091C602F80185835BC1C114D10431F054
:103BB0005F3F31F481E04F3F19F403C081E001C061
:103BC00080E080FD03C081E08F2502C080E090E0AE
:103BD000F82FF170EF2E80FF1CC080918F02209192
:103BE000900236E0821709F418C190E0389FF00186
:103BF000399FF00D1124EF56FD4F6181561306C019
:103C00006081461303C06281F61203C0019687707B
:103C1000E9CFEF2CFF2009F423C18091C602816017
:103C20008093C60262C0561306C0491304C0F11047
:103C300002C0F801A7C04D875E87FF867C2DD98A18
:103C4000C88A6F2D89890E94571C882399F1FF200B
:103C500089F12091C602822F82958F7090E00297A1
:103C600074F08091C1029091C20298878F83198667
:103C7000DB86CA862C87CE0107960E944D1986E006
:103C8000F801A1ECB2E001900D928A95E1F70E9453
:103C9000031D0E94F51C11C0561749F14D875E8720
:103CA000FF867C2DD98AC88A6F2D89890E94571C6E
:103CB00081112CC0C8010E944D19EE24E394D0C09C
:103CC000282F207F49F77C2DD98AC88A6F2D8989B2
:103CD0000E94B51C81EC92E00E944D1986E0F5012E
:103CE00011928A95E9F70E94F51CE12CB9C049139D
:103CF000D5CFF110D3CFF8018583C8010E944D19AB
:103D000086E0F50111928A95E9F7AAC0FF2091F2A9
:103D10002091C602822F82958F7090E002970CF45A
:103D2000AECF8091C1029091C2029A8389831B8297
:103D3000DD82CC822E83CE0101969FCFE83CF10537
:103D400008F04BC0EF2CFF2009F4B4CF561330C05D
:103D500049132EC02091C60220FD21C0822F8295DA
:103D60008F70482F50E041155105C9F0F8012583A7
:103D70004F30510541F08F5F982F9295907F822FA1
:103D80008F70892B8583C8010E944D1986E0F80148
:103D9000A1ECB2E001900D928A95E1F72AC086E08D
:103DA000F801A1ECB2E001900D928A95E1F758C0BC
:103DB0004D875E87FF867C2DD98AC88A6F2D8989B9
:103DC0000E94571C81115BCF8091C6028160809355
:103DD000C602C8010E944D1943C07C2DD98AC88AE9
:103DE0006F2D89890E94B51C86E0F50111928A9594
:103DF000E9F70E94F51C34C0FF2009F45BCF4D8722
:103E00005E87FF867C2DD98AC88A6F2D89890E949A
:103E1000571C882309F44ECF32CF7C2DD98AC88A0B
:103E20006F2D89890E94A721292F22952F7022307A
:103E300028F49F7039F0811105C00BC0243028F49C
:103E40009F7049F4805E883020F0C8010E944D19AF
:103E50009E2CE92C05C0F8019581907F99F7F9CF48
:103E60008E2D61960FB6F894DEBF0FBECDBFDF91E9
:103E7000CF911F910F91FF90EF90DF90CF90BF9067
:103E8000AF909F9008951F93CF93DF93CDB7DEB788
:103E90002C970FB6F894DEBF0FBECDBF4F83588767
:103EA00069877A878B879C87CE0107960E946F1D52
:103EB0008823D1F09F8188852A853B85232B31F08B
:103EC0008F3F31F481E09F3F19F403C081E001C0CE
:103ED00080E080FD47C04F81588569857A858B8554
:103EE0009C850E94C41C3EC086E0FE013796DE0120
:103EF000119601900D928A95E1F7FF81E8856A8518
:103F00007B856115710531F0EF3F31F481E0FF3FB2
:103F100019F403C081E001C080E080FD23C020913E
:103F2000900230E0C90101968770992740918F0275
:103F300050E084179507F1F1F983EA837D836C8360
:103F400096E0929FD001939FB00D1124AF56BD4FC4
:103F5000FE01319601900D929A95E1F780939002BF
:103F60000E94D41C16E080918F02909190028917D4
:103F700071F1189FC00111248F569D4F0E946F1D33
:103F8000882329F1E0918F021E9FF0011124EF5642
:103F9000FD4F4081518162817381848195810E94AE
:103FA000C41C80918F0290E00196877099278093BE
:103FB0008F02D9CF0E9449191092900210928F025D
:103FC000E1ECF2E086E0DF011D928A95E9F72C969C
:103FD0000FB6F894DEBF0FBECDBFDF91CF911F911A
:103FE0000895DF92EF92FF920F931F93CF93DF9389
:103FF000FC01892B09F488C0E12CF12CDD24D39439
:10400000EF0121968491853709F460C058F4843714
:1040100008F04EC0843008F068C08130D1F08230A2
:1040200071F172C0883709F45BC050F4863709F427
:1040300053C0873709F068C08E2D0E94DD2252C020
:104040009CE7980F903708F05FC08F770E940119A6
:104050004EC08F010E5F1F4FFE01849190E2980FBA
:10406000983050F48770FD2D01C0FF0F8A95EAF754
:104070008F2F0E94E32215C00E94961814C08F0152
:104080000E5F1F4FFE01849190E2980F983068F404
:104090008770FD2D01C0FF0F8A95EAF78F2F0E94D0
:1040A000E9220E940A23E80122C00E940119FBCFE5
:1040B000CF010296FE01C491CC2361F0EFE9FFE04D
:1040C0003197F1F700C00000C150F6CFCF01029642
:1040D000FE01F490EC010BC00E94CD22E82E07C037
:1040E0000E94E0220E940A2302C00E9496188F2D8F
:1040F000882341F0EFE9FFE03197F1F700C00000BD
:104100008150F6CFFE017CCFDF91CF911F910F91AF
:10411000FF90EF90DF9008956093470370934803FA
:104120008093490390934A030C9458230895609315
:104130004B0370934C0380934D0390934E030C9468
:1041400057230F931F9300914B0310914C03209121
:104150004D0330914E03602B712B822B932B609378
:104160004B0370934C0380934D0390934E031F9128
:104170000F910C9457230F931F9300914B031091B1
:104180004C0320914D0330914E0360237123822311
:10419000932360934B0370934C0380934D03909350
:1041A0004E031F910F910C9457230F931F9300916F
:1041B0004B0310914C0320914D0330914E03602727
:1041C00071278227932760934B0370934C0380934E
:1041D0004D0390934E031F910F910C94572360E071
:1041E00070E0CB010C948C200F931F9341E050E0C2
:1041F00060E070E08A019B0104C0000F111F221FC4
:10420000331F8A95D2F7C901B8011F910F910C9401
:104210008C200F931F9341E050E060E070E004C0F9
:10422000440F551F661F771F8A95D2F78091470369
:1042300090914803A0914903B0914A038A019B01E0
:10424000082B192B2A2B3B2BC901B8011F910F9169
:104250000C948C200F931F9341E050E060E070E0DD
:1042600004C0440F551F661F771F8A95D2F74095EB
:104270005095609570958091470390914803A09167
:104280004903B0914A038A019B01082319232A2379
:104290003B23C901B8011F910F910C948C200F93FF
:1042A0001F9341E050E060E070E004C0440F551FF0
:1042B000661F771F8A95D2F7809147039091480334
:1042C000A0914903B0914A038A019B01082719274D
:1042D0002A273B27C901B8011F910F910C948C200C
:1042E0000F931F93009147031091480320914903B6
:1042F00030914A03602B712B822B932B1F910F91CE
:104300000C948C200F931F93009147031091480346
:104310002091490330914A03602371238223932320
:104320001F910F910C948C200F931F9300914703C2
:10433000109148032091490330914A036027712767
:10434000822793271F910F910C948C2008958F92B0
:104350009F92AF92BF92DF92EF92FF920F931F93C3
:10436000CF93DF9300D000D01F92CDB7DEB76B8321
:104370007C838D838A018C819D81892B31F01F3F45
:1043800031F481E04F3F19F403C081E001C080E0C7
:1043900080FF03C080E090E04DC08B818823D1F185
:1043A0008090470390904803A0904903B0904A033F
:1043B00080914B0390914C03A0914D03B0914E031B
:1043C000882A992AAA2ABB2A8FE1E82EF12CD50146
:1043D000C4010E2C04C0B695A795979587950A94AD
:1043E000D2F780FD06C081E0E81AF10880F7D12CF1
:1043F00007C0DE2CB8018E2D0E946606019799F346
:1044000088E0189FF0011124E953FD4FE00FF11DE2
:10441000D08209C088E0189FF0011124E953FD4FB4
:10442000E00FF11DD08009831A8369817A818D2D77
:104430000E9466060F900F900F900F900F90DF91E3
:10444000CF911F910F91FF90EF90DF90BF90AF90B1
:104450009F908F90089590911401992379F19091F4
:104460001501992359F1982F9695969596959F3118
:10447000A1F0E0911601F0911701E90FF11D87708D
:1044800021E030E0A90102C0440F551F8A95E2F7F0
:10449000CA019181892B818308959091720390FFC5
:1044A00029C01F928F9386E897E09F938F930E9475
:1044B0005D060F900F900F900F90089520911601B8
:1044C00030911701F90132969FEF40E05191851725
:1044D00089F09F3F19F4511101C0942F4F5F4E3165
:1044E000A9F79F3F39F0F901E90FF11D97FDFA9502
:1044F00082830895089590911401992381F19091F8
:104500001501992361F1982F9695969596959F316F
:10451000A9F0E0911601F0911701E90FF11D8770E4
:1045200021E030E0A90102C0440F551F8A95E2F74F
:10453000CA018095918189238183089590917203A6
:1045400090FF1CC01F928F9388E697E09F938F93F4
:104550000E945D060F900F900F900F900895E091CC
:104560001601F09117019F01225E3F4F928189133E
:1045700001C012823196E217F307C1F7089581E076
:1045800090E0E0911601F0911701E80FF91F1082F9
:10459000019680329105A9F70895809171030895DD
:1045A00090917103892B8093710308958095909168
:1045B0007103892380937103089580937103089593
:1045C00010927103089590917003892B809370036A
:1045D00008958095909170038923809370030895C6
:1045E00010927003089580934F03089510924F0323
:1045F00008958091160190911701FC0131969C015C
:10460000205E3F4F80E0919191118F5FE217F30799
:10461000D1F70895E0911601F0911701809171038F
:104620008083E0911601F0911701908180917003D1
:10463000892B808380914F03882361F0E0911601DC
:10464000F09117019081892B80830E94F9228111BA
:1046500010924F0380911601909117010C94CD1682
:10466000909335018093340108958295982F937328
:1046700044E0949F900111248C7C86958695282B8C
:10468000822F8575880F2A7A2695822B08950895A2
:10469000CF93DF9300D000D01F92CDB7DEB70F903D
:1046A0000F900F900F900F90DF91CF910895089584
:1046B00008950C94171880E0089583B7817F8C606B
:1046C00083BF83B7816083BF7894889583B78E7FDB
:1046D00083BF0895CF930E944E180E947C0A0E94C7
:1046E0004F18C0E08C2F0E945F0A811104C0CF5F79
:1046F000C031C1F701C081E0CF9108950E94650AE1
:104700000C9449191F920F920FB60F9211248F9398
:104710009F93AF93BF938091730390917403A09183
:104720007503B09176034196A11DB11D809373036B
:1047300090937403A0937503B0937603BF91AF91E8
:104740009F918F910F900FBE0F901F90189582E050
:1047500084BD93E095BD9AEF97BD80936E00089558
:104760002FB7F8948091730390917403A09175030F
:10477000B09176032FBF08952FB7F894609173031B
:104780007091740380917503909176032FBF089503
:104790009C014FB7F8948091730390917403A0919A
:1047A0007503B09176034FBF821B930B08951F9240
:1047B0000F920FB60F9211248F939F93AF93BF93D5
:1047C0008091730390917403A0917503B091760367
:1047D0000196A11DB11D8093730390937403A09360
:1047E0007503B0937603BF91AF919F918F910F9016
:1047F0000FBE0F901F9018950E945115F89487E7EF
:1048000097E7909301088093000887E090EBDC0124
:104810008093850390938603A0938703B0938803C6
:104820009CE088E10FB6F894A895809360000FBED5
:1048300090936000FFCF80E090E008950895CF93BB
:10484000C82F1F928F938AEA97E09F938F930E94BD
:104850005D0681E090E0A0E0B0E0BC01CD0104C0C5
:10486000660F771F881F991FCA95D2F70E9497205D
:104870000F900F900F900F90CF910C944919CF93F8
:104880008732A8F58E3108F02BC1803109F49FC022
:10489000F8F4873009F464C0A8F4863009F024C124
:1048A00080917203817F8E7F809372038FEA97E0FD
:1048B0000E94C40582E99AE00E94C40581E08093C9
:1048C00077034CC08B30F1F18E3009F46CC00CC111
:1048D000863109F4B0C020F4813109F4EDC004C17F
:1048E000893109F491C08B3109F449C0FDC0883386
:1048F00049F150F4893209F4F1C0853309F4EEC06E
:10490000873209F0F1C0EAC0833409F4E7C028F423
:104910008A3308F4E9C08953E4C0883409F0E4C05C
:104920000E94491981E89AE00E94C4052FEF83EDA7
:1049300090E3215080409040E1F700C000000E94C9
:10494000FC230CC08AEC97E05CC088E69AE00E94E9
:10495000C40580917203816080937203C1E0C9C075
:1049600080917203C82FC17080FFEFCF84E79AE077
:104970000E94C40580917203817F8E7F3DC090911B
:10498000720391FBCC27C0F981E0C827892FC0FBB7
:1049900081F980937203CC2319F08BE59AE027C04C
:1049A0008DE49AE02EC09091720392FBCC27C0F95F
:1049B00081E0C827892FC0FB82F980937203CC2342
:1049C00019F08EE39AE013C08EE29AE01AC090913B
:1049D000720393FBCC27C0F981E0C827892FC0FB65
:1049E00083F980937203CC2351F082E29AE00E9413
:1049F000C405809172038160809372037AC085E15F
:104A00009AE00E94C405AACF86E09AE00E94C405FD
:104A100080EE99E00E94C40588E999E00E94C405EF
:104A200080E799E00E94C40584E299E00E94C405F1
:104A300088EF98E0E6CF8AEE98E00E94C4050E94D5
:104A4000C1161F928F9380ED98E09F938F930E94E1
:104A50005D06809114011F928F9389EB98E09F93DC
:104A60008F930E945D06809177021F928F9386EA52
:104A700098E09F938F930E945D06809115011F928D
:104A80008F9383E998E09F938F930E945D060E9425
:104A9000BC239F938F937F936F938CE798E09F93B2
:104AA0008F930E945D068DB79EB746960FB6F89419
:104AB0009EBF0FBE8DBF52CF0E944919C0911501F4
:104AC00081E0C827C0931501CC2329F082E798E044
:104AD0000E94C4050EC087E698E093CF80E001C035
:104AE0008D510E941F243ACF85E698E00E94C405AC
:104AF000C0E08C2FCF91089580E008950C947C2520
:104B0000CF93C82F80917703882319F0813059F013
:104B100042C0E0911601F09117018081823261F06C
:104B20008434D9F509C0E0911601F0911701808114
:104B3000823211F0843461F48C2F0E947E25811121
:104B400004C08C2F0E943F2424C081E090E021C04B
:104B50008C2F0E947C2581111BC0C43189F018F470
:104B6000CB3029F010C0C93259F0C83361F48FEA54
:104B700097E00E94C40586EA97E00E94C40508C039
:104B8000109277030CC084EA97E00E94C40507C026
:104B900081E0817006C01092770380E002C080E05F
:104BA000F8CFCF910895EE0FFF1F0024001C0BBE1D
:0C4BB0000790F691E02D0994F894FFCFD7
:104BBC000080FFFF0556010000FF790EE60E7C0E0B
:104BCC00B10E7D0E0101500340362239D0069A06F3
:104BDC0078063F06CB05E405FD051D060000100018
:044BEC0008000400B9
:106800008800EA44E944E244040005000600070069
:10681000080009000A000B000C000D000E000F001C
:1068200010001100120013001400150016001700CC
:10683000180019001A001B001C001D001E001F007C
:10684000200021002200230024002500260027002C
:10685000280029002A002B002C002D002E002F00DC
:10686000300031003200330034003500360037008C
:10687000380039003A003B003C003D003E003F003C
:1068800040004100420043004400450046004700EC
:10689000480049004A004B004C004D004E004F009C
:1068A000500051005200530054005500560057004C
:1068B000580059005A005B005C005D005E005F00FC
:1068C0006000610062006300640065A185006700EC
:1068D000680069006A006B006C006D006E006F005C
:1068E0007000710072007300890087008A008B00BD
:1068F000E000E100E200E300E400E500E600E7007C
:106900000100010001000100EA4401000100E2442D
:106910000100010001000100460001004A004B0097
:10692000010001004700480001000100E9440100A6
:106930000100010001000100010001003A003B00DC
:106940003C003D003E003F0040004100420043004B
:10695000010035004C0039000100440045005200A0
:1069600049000100010050004F0029004D004E0079
:1069700051000100010001000100010001000100BF
:1069800001000100010001000100010001000100FF
:1069900001000100010001000100010001004D00A3
:1069A0004A004E004B0001000100010001000100FF
:1069B00001000100010001000100010001000100CF
:1069C00001000100010001000100010001000100BF
:1069D00001000100010001000100010001000100AF
:1069E0000100010001000100490001000100010057
:1069F000010001000100010001000100010001008F
:00000001FF
